:02000000040AF0
:080008009F0C0200080C060029
:10001000740A000000000000110C27000000E70235
:100020000E0A00084B0C2800F90C29000000E90218
:10003000160AE802140A000866061C0A09090909DA
:1000400066061C0A6607220A09090909090909093D
:1000500009090909090909090909090966071C0AA1
:10006000090909090909090909096607770A090936
:100070000909090909096607840A090909096607BE
:10008000000809090909090909096607840A770AA4
:100090006606480A090909096606480A66074E0AFB
:1000A00009090909090909090909090909090909C0
:1000B000090909096607480A090909090909090915
:1000C00009096607770A090909090909090966077B
:1000D000840A090909096607870A0909090909093A
:1000E00009096607840A770A070C2600480A010CEA
:1000F00026001209000C26001209010C2600120924
:10010000000C26001209480A010C2600480A030CBC
:10011000260012091C09010C260012091C09030CF7
:10012000260012091C09010C260012091C09030CE7
:10013000260012091C09010C260012091C09030CD7
:10014000260012091C0912091C0912091C091209AE
:100150001C0912091C0912091C0912091C0912099F
:100160001C0912091C0912091C0912091C0912098F
:100170001C0912091C0912091C0912091C0912097F
:100180001C0912091C0912091C0912091C0912096F
:100190001C09040C26001209120912091209000C8C
:0E01A000260012091209120912091C09C90AC7
:021FFE00E90FE9
:00000001FF
